:10000E004150545832410057494445312000574918
:05001E00444532200002
:102B990025E0FF900297E02402F582E43401F583F1
:102BA90022EFF0900297E004F022EFF0900296E015
:102BB90004F0A3E004F0227B017A017902900183F9
:102BC900E0FD227C007D0A120303ED2430229002ED
:052BD9009BE025E02255
:102BDE00120B67122BC01226B4122BC0121B797F58
:102BEE00C01232CDE4FF1232CDE4900295F0900186
:102BFE0083E0FF900295E0FEC39F501374022E12E5
:102C0E002BA2E0FF1232CD900295E004F080DF7F20
:042C1E00C00232CDF1
:100B6700E4900297F0900296F0900296E090000EC3
:100B7700936008122B99122BB380EE122B9C746092
:100B8700122BABE4A3F0A3F0A37408F0120E6BEFE3
:100B97006020120E6BEF122B99EFF090029AE0048F
:100BA700F07006900299E004F0122BACA3E004F079
:100BB70080DA900298E0C394065028E4900296F0F9
:100BC700900298E0FFC374069FFF900296E0C39FD0
:100BD7005011A3122B9F7440122BAB900296E00486
:100BE700F080DD7F0F7E0012315690029BEFF07F81
:100BF700107E00123156EF24FE602804706D122B10
:100C0700D744E0122B9B122BAAE4900296F0900295
:100C170096E0900015936008122B99122BB380EE83
:100C2700020C6B122BD744E0122B9B122BAAE490D9
:100C37000296F0900296E0900015936008122B99A7
:100C4700122BB380EE122B9C7462122BABE4900232
:100C570096F0900296E090001C936008122B991270
:100C67002BB380EE122B9C74638009122BD744613F
:100C7700122B9BEF122BAB122B9C7403122BAB1274
:100C87002B9F74F0122BAB7F117E00123156122B63
:100C97009C122BAAE4900296F0900296E02418F595
:100CA70082E43403F583E0FF6008122B9C122BB318
:100CB70080E77F127E00123156122B9C122BAAE47A
:100CC700900296F0900296E0240EF582E43403F544
:100CD70083E0FF6008122B9C122BB380E77F137E03
:100CE70000123156122B9C122BAA9002FFE0FAA396
:100CF700E0FB7C007D64FFAE02120303EF24301299
:100D07002B9B122BAA7C007D0AAF03AE02120303B2
:100D1700122BCCFF122B9F122BAA9002FFE0FEA3EF
:100D2700E0FF122BCC122B9B122BAA122B9F742F96
:100D3700122BAB90030AE0FF75F064842430FE1297
:100D47002B9CEE122BABEF75F00A8475F00A84E545
:100D5700F02430FF122B9F122BAA90030AE075F0A4
:100D67000A84E5F02430122B9B122BAA122B9F74B6
:100D77002F122BAB122B9F7441122BAB122B9F748C
:100D87003D122BABE4900296F0900296E0FFC394DD
:100D970006501974032FF582E43403F583E0122B10
:100DA7009B122BAA900296E004F080DD900299E452
:100DB700F0A37440F0120E77EF601B120E77122B20
:100DC7009CEFF090029AE004F07006900299E0041C
:100DD700F0122BAC80DF122B9C7420122BAB122C41
:100DE700A9E4900296F0900296E0243FF582E4345D
:100DF70003F583E0FF6008122B9C122BB380E712E8
:100E07001393EF64017026122B9C7420122BABE412
:100E1700900296F0900296E02435F582E43403F5CB
:100E270083E0FF6008122B9C122BB380E7120E831E
:100E3700300826122B9C7420122BABE4900296F0FC
:100E4700900296E024D6F582E43402F583E0FF6051
:100E570008122B9C122BB380E7900297E090018336
:030E6700F07F0118
:100E6A0022900299E0FEA3E0FF12315622900299E5
:090E7A00E0FEA3E0FF1231562254
:102B0600E0FAA3E0FBFFAE02120303EF2430FF90CE
:102B1600029FE02435F582E43403F583EFF090025A
:102B26009FE004F0227C00AF03AE021203037C0098
:102B36007D0A120303ED22E02435F582E43403F521
:0D2B46008322E0FAA3E0FB7C007D0AFF2261
:10139300122F36EF7002FF227FCC1200267F4412F9
:1013A300002630A0FD122F36EF7002FF227FCC12F1
:1013B30000267FBE120026122FD490033DE4F0A333
:1013C300EFF0122FD490033BE4F0A3EFF0E490028C
:1013D3009FF090029FE0FFC39406500C74352F12C8
:1013E3002B40E4122B2380EA90033BA3E0FF30E77A
:1013F3001DD20BFE90033EE02400FF90033DE03E30
:10140300FEEFF4FFEEF4FEEF2401FDE48012C20BC5
:1014130090033CE0FE90033EE02400FD90033DE09A
:101423003EFCE41201F1E4FBFA7920783F12004616
:1014330012022A9002A0EEF0A3EFF0E490029FF0D4
:10144300300B08122B3D742D122B23C39002A1E005
:1014530094649002A0E09400500C122B48AE021248
:101463000303EF0214CCC39002A1E094E89002A01E
:10147300E09403502C7C007D64122B067D0A122B12
:101483002B2430FF122B18122B3D742E122B23A367
:10149300E0FEA3E0FF122B342430FF90029F0214DE
:1014A300E6C39002A1E094109002A0E0942750417B
:1014B3007C037DE8122B067D64122B2B2430FF1254
:1014C3002B18A3122B48122B2F122B12122B3D7405
:1014D3002E122B237C007D0AAF03AE02120303ED11
:1014E3002430FF122B18122B3D7443122B237F0140
:0314F300227F0055
:0114F60022D3
:07310B00123112D2A07F0176
:10311200AE071FEE600D000000000000000000007E
:043122000080ED221A
:102F3600D2D7C2A07FF01231127FF0123112D2A086
:102F46007F3C123112A2A07FF01231127FB41231EF
:0A2F56001220D7037F01227F002222
:102FD400E4FDFCEDC313FDC2A07F0112310B30A050
:102FE40004ED4480FD7F3C1231120CECB408E4AFD4
:012FF40005D7
:012FF50022B9
:02002600AD0724
:10002800E4FCC2A07F01123112EDC313FD92A07F40
:090038003C12310B0CECB408E998
:01004100229C
:101E7600EF2430F09002CBE0FCA3E0FDA3E0FEA34C
:101E8600E022FFEE3395E0FDFCE0F8A3E0F9A3E0E5
:101E9600FAA3E022FFE4FAF9F8122C22AC00AD0115
:101EA600AE02AF039002CB0204E4F00B74D62BF51E
:101EB60082E43402F58322A804A905AA06AB07E04A
:101EC600FEA3E0FFEE3395E0FDFC222FFFEA3EFE87
:101ED600E93DFDE83CFC2212036E78101204BD9029
:101EE60002AB1204E49002AB221204BD9002A702D8
:101EF60004E4EF2402FFE43EFEE43DFDE43C22F868
:101F0600E0FEA3E0FFE4FCFD12036E780F22FF1251
:0F1F16002C22EF243022FB12036E780C0204BD44
:1021AE00121EAA7BA07A8679017800121E7AFF127F
:1021BE002C229002E5121E76FF7BA07A867901789A
:1021CE0000121E9FE47B107A27F9F8121E7AFF1276
:1021DE002C229002D0121E76FFE47B107A27121E5C
:1021EE009DE47BE87A03F9F8121E7A121F1490020E
:1021FE00EF121E79FFE47BE87A03121E9DE47B64E6
:10220E00FAF9F8121E7A121F149002F0121E797B40
:10221E0064121E9AE47B0AFAF9F8121E7A121F143F
:10222E009002CF121E797B0A121E9A9002CBA3A3A4
:09223E00A3E024309002D1F0224B
:0D320A00E4FF9002CBE004F00FEFB46EF58E
:013217002294
:0E321800E4F5D875F9DCF5E9D2DE30DFFD22F1
:0F31BF00D2A4D2A312320AC2A412320AC2A3228D
:0C329300C2A4D2A312320AD2A402320A52
:0E322600A20B92A4D2A312320AC2A302320A51
:10316D00D2A312320AA2A430A404C2088002D2084B
:06317D00C2A312320A2277
:0230B700AE0762
:1030B900E4FDEE25E0FE92A4D2A312320AC2A312C5
:0A30C900320A0DEDB408EB02316D80
:10301800E4FED2A4FDEE25E0FED2A312320AA2A459
:10302800E4334EFEC2A312320A0DEDB408E7AF0630
:013038002275
:022D5E00AC07C0
:102D60001231BF7FEE1230B7AF041230B71231BF4D
:102D70007FEF1230B7123018AC07C20B1232261296
:102D80003018AD07D20B123226123293123218AF1E
:052D900004EFFEEDFF61
:012D9500221B
:103039001231BF7FEE1230B77FF41230B77F2E12F4
:1030490030B71232931232187FF6122D5E121ECA51
:013059002254
:102F60007F007E007D007C001231BF7FEE1230B703
:102F70007FF41230B77F341230B712329312321806
:082F80007FF6122D5EE4FDFC5A
:012F88002226
:102247007FAA122D5E9002F3EEF0A3EFF07FAC129F
:102257002D5E9002F5EEF0A3EFF07FAE122D5E90AB
:1022670002F7EEF0A3EFF07FB0122D5E9002F9EEC9
:10227700F0A3EFF07FB2122D5E9002FBEEF0A3EF1A
:10228700F07FB4122D5E9002FDEEF0A3EFF07FB663
:10229700122D5E9002D2EEF0A3EFF07FB8122D5E02
:1022A7009002D4EEF0A3EFF07FBA122D5E9002E613
:1022B700EEF0A3EFF07FBC122D5E9002E8EEF0A3E4
:1022C700EFF07FBE122D5E9002EAEEF0A3EFF02250
:100E830012303990029F1204E4122F609002A312D1
:100E930004E49002FDE0FEA3E0FBAA0690029F1289
:100EA3001E7DC39BFBEE9AFAED9400F9EC9400903F
:100EB30002FB121F05121EEF9002E8121EC5780BEB
:100EC3001204D1C004C005C006C007A3E0FEA3E01E
:100ED3009002A7121E882FFBEA3EFAE93DF9E83C8F
:100EE300F8D007D006D005D004122C22121EE5122A
:100EF3001E7DFF9002A7121E8F121ED19002AF1209
:100F030004E49002AF121E7D2408121EFBFC780439
:100F13001204BD1221AE9002F0E09002E0F09002C4
:100F2300CFE09002E4F09002D1E09002ECF0900266
:100F3300AF121E7D2460FFEE34F0FEED34FFFDECB6
:100F430034FFFCA31204E49002B3121E7DFFA80435
:100F5300A905AA06121F1C9002D4121EBD12036E0D
:100F6300780B121EEF9002F5E0FEA3E09002B3129D
:100F73001E88FB12036E780B121EE2121E7DFF9079
:100F830002A7121E8F121ED19002B71204E4900220
:100F9300F3121EC5E47B04FAF9F812036E9002B74C
:100FA300121E8F121ED1121EF8FCE47B04FAF9F80C
:100FB300122C229002BB1204E49002F7121EC59079
:100FC30002B3121E8FFB12036E780D121EEF9002F6
:100FD300B3121E7DFF9002B3121E8F121F1C9002CC
:100FE300D2121EBD121EDD121E7DFF9002A7121E1D
:100FF3008F121ED1121EF8FC78021204BD9002B7A4
:101003001204E49002B7121E7D2400FFEE34801216
:101013001EFEAB07AA06A9059002F9121F051204CA
:10102300AA9002C31204E49002A3121E7DFFC0041F
:10103300C005C006C0079002BB121E7DFBAA06A90D
:1010430005A804D007D006D005D004C3EF9BFFEE5C
:101053009AFEED99FDEC98FCE47B507AC3F9F81203
:10106300036E9002C71204E4E4FFFEFD7C8090024D
:10107300C7121E8FFBC3120499501EE47F02FEFDAC
:10108300FC9002C7E0F8A3A3A3E012036E9002C38F
:10109300121E8FFB1203F980189002C3121E8FFBDE
:1010A300A3121E7DFF1203F9E47B02FAF9F812037F
:1010B3006E9002BF1204E49002BF121E7DFF7808F7
:1010C3001204BDC004C005C006C0079002BF121EB3
:1010D3007DFF78081204BDD003D002D001D00012E6
:1010E300036E121EF2E47FDE7E0BFDFC9002A7125C
:1010F3001E8FFB12036E7810121EEF7F437EE37D7B
:10110300FF7CFF9002BF121E8FFB121EDD121E7D9D
:10111300FF9002A7121E8F121ED1EF24CFFFEE34D1
:101123000E121EFEFC78041204BD9002BF121E8F25
:10113300121ED11221AE9002E5E0FF9002EEF09074
:1011430002D0E0FE9002F2F09002EFE0FD9002E1A7
:10115300F09002F0E0FC9002EDF09002CFE0F99005
:1011630002F1F0E4FB24D6121EB5EF121EB0EE120C
:101173001EB0ED121EB0EC121EB0742E121EB0E99A
:0F118300121EB07470F074D62407121EB5E4F07B
:01119200223A
:1024FC001203F9EB2430FF9002A3E0243FF582E4B1
:10250C003403F583EFF09002A3E004F0E0243FF5F0
:10251C0082E43403F583227F07122D96E4FCFD122E
:10252C0001ECE4FBFA79407840120046E4FBFA79BE
:10253C0080784412014FE4FBFA227B0AFAF9F890F6
:10254C00029FE0FCA3E0FDA3E0FEA3E0FF2279489C
:0F255C00784312004602022A900293E094012273
:0D326C00439180439280439D8075BCA02259
:102D9600E4F5BDF5BEE5BC54E044084FF5BC0000C3
:102DA60000007DFAE5BC30E41753BCEFAFBDEF750C
:102DB600F004A4FFACBEEC7A002FFFEA35F0FE2249
:062DC600DDE27E037FFF49
:012DCC0022E4
:102CA90012252379A0784112255E90029F1204E42F
:102CB900E49002A3F01225461203F9E47B0AFAF91B
:102CC900F81224FC742EF09002A3E004F0E412251B
:102CD900461224FC7456122511E4F09002A3E00474
:012CE900F0FA
:012CEA0022C7
:1027E80012252312255A900293EEF0A3EFF0C3941A
:1027F8009AEE940140047F068042C3900294E094CC
:102808007C12256440047F058032C3900294E094D2
:102818005E12256440047F048022C3900294E094F1
:102828004012256440047F038012C3900294E09410
:0F2838003112256440047F0280027F01122FB00D
:01284700226E
:1025DA00E490029BF0A3F0A3F07F07122D96E4FC8F
:1025EA00FD9002971204E490029712254EE41225F8
:1025FA002B12255A9002931204E4900293A31225F7
:10260A005390029CE02FF090029BE03EF090029DD6
:10261A00E004F0E0C3940A40C090029BE0FEA3E00D
:10262A00FF7C007D0A12030390029BEEF0A3EFF0F9
:0D263A00C39431EE940150037F01227F0014
:012647002270
:102FB000900295EFF0900295E0FF14F0EF6014C2DC
:102FC000907F037E0012307BD2907F037E00123010
:042FD0007B80E222FE
:10307B00EF4E6019EF1FAC0670011E4C600FE4F5AC
:0E308B00D875F94CF5E9D2DE20DFE980FB2292
:0D327900D2C2D280D290D282D283D28122E2
:1030D3001226481232C31230991228A612295D1201
:0C30E30021111225DABF01EBC20980E7C1
:1030990020961A7F017E0012307B209610B2843070
:0E30A90096FD7F017E0012307B3096F32222CE
:102EB5002096277F017E0012307B20961D7F011210
:102EC50014F7C2C2C290C282C2813096FD7F017ED4
:0B2ED5000012307B3096F375C72022FE
:03000300022903CC
:10290300C0E0C0F0C083C082C0D075D000C000C09A
:1029130001C002C003C004C005C006C00720B21F27
:102923007F017E0012307B20B215B20930B2FD7FE9
:10293300017E0012307B30B2F330090375C720D01B
:1029430007D006D005D004D003D002D001D000D0E8
:0A295300D0D082D083D0F0D0E03263
:0A32C300200906123234758702223A
:0E323400C294C284C2C0D2B6D2B7123279227E
:10264800123234D209D2C01232DE75BBFFE4F591E2
:10265800759220F5B375B40143B70243B80243B786
:1026680010C2C2C280C290C282C283C2817F0AFEE7
:1026780012307B12327912313E122EB512326C12A0
:1026880031CE1232E5122247121393121393122FEE
:1026980089C28CE490034DF0C28CC28D758C4CF5C8
:0C26A8008AD28CD2A8D2A9D2AF0227E8B7
:03000B00022A0DB9
:102A0D00C0E0C0F0C083C082C0D075D000C000C08F
:102A1D0001C002C003C004C005C006C007C28CC2FD
:102A2D008D758C4C758A00D28C90034DE004F0E0CE
:102A3D00D394144005E4F01223F7D007D006D00547
:102A4D00D004D003D002D001D000D0D0D082D0831A
:052A5D00D0F0D0E032D2
:10162F00504F5745523A200020202054454D503AF4
:10163F002000202D2D2D2D2D2000202020507265D3
:10164F0073737572653A2000200D0A0D0A0041541C
:10165F002B48454C503D310D0A0041542B44454D0C
:10166F004F3D310D0A0041542B43414C4C3D000D71
:10167F000A0041542B535349443D0041542B5449C4
:10168F004D453D0041542B424541434F4E3D000DCA
:10169F000A0D0A002A2A2A2041505253203531546C
:1016AF007261636B2058324128424C41434B424F89
:1016BF0058292032303134303930352042483454B3
:1016CF00445620202A2A2A200D0A004E4F43414C0F
:1016DF004C00333133342E35354E00003132303239
:1016EF00302E3636450041505253203531547261F9
:1016FF00636B2058324120210000000000000000E1
:10170F0000000000312C3433382E353030302C347B
:10171F0033382E353030302C302C332C3000000045
:10172F000000312C3134342E363430302C313434F7
:10173F002E363430302C302C332C302C300000002F
:1027870090029CE0FEA3E0FFE4FD1230EFE004F0CE
:102797002290029BA3E02400F582E43400F5832213
:1027A70090029BE0FEA3E0FF2290029CE004F0224F
:1027B70090029CE0FEA3E0FF2290029BE004F0223F
:1027C70075C65A75C6A52290029CE4F0A322ECF5C3
:1027D700C3AF058FC422F0A3EFF0C3940AEE9400B1
:0127E70022CF
:1004F000E490029DF0A3F090029BF0A3F090029D87
:10050000E0FEA3E0FF123156122798EFF090029E12
:10051000E004F0700690029DE004F090029CE0047C
:10052000F070031227C0C390029BE0940140CE7B81
:10053000FF7A1679A3122E5D122CA97BFF7A167909
:100540002F122E5D7B017A03793F122E5D7BFF7A9D
:10055000167937122E5D121393BF01087B017A03BF
:10056000793580067BFF7A167941122E5D7BFF7A02
:10057000167949122E5D120E833008087B017A022B
:1005800079D680067BFF7A167941122E5D7A16792C
:100590005712082A7A16795D122E5D7BFF7A16793A
:1005A00069122E5D7BFF7A167975122E5D90029B83
:1005B000E4F0A37408F0122798E0FF600A1208150F
:1005C00070F41227C080EF1208097A167981122E72
:1005D0005D90000FE0FF7E0090029BEE1227DD127F
:1005E00027A77C007D0A5002800A1207D71227A78E
:1005F0007C007D0A12081F1208097A16798A122EC9
:100600005D900000E0FEA3E07C002400FFEC3EFED5
:1006100090029B1227DD500B90029BA3E02430FF39
:100620001232CD1227A7D39409EE940040047D0125
:1006300080027D00C3EF9464EE940050047F01803B
:10064000027F00EF5D60031207A31227A7D3946314
:10065000EE940040047D0180027D00C3EF94E8EE3B
:10066000940350047F0180027F00EF5D600D12272C
:10067000A77C007D641207D71207A31227A7D39483
:10068000E7EE940340047D0180027D00C3EF9410E7
:10069000EE942750047F0180027F00EF5D60061218
:1006A00007431207E91227A7D3940FEE94274014AB
:1006B0007C277D101203031207E91207437C007D9B
:1006C0000A12081F7A16797E12082A7A167993126E
:1006D0002E5D900010E0243012083C9000111207AB
:1006E000F87420F0122798E0FF600A12081570F4E1
:1006F0001227C080EF7F2C1232CD9000121207F823
:100700007430F0122798E0FF600A12083270F41279
:1007100027C080EF7F2C1232CD900013E012083CEE
:1007200090029BE4F0A37440F0122798E0FF600A67
:1007300012083270F41227C080EF7BFF7A16799E80
:03074000022E5D29
:1007430090029BE0FEA3E0FF7C037DE81203037CA1
:10075300007D0A120303ED2430FF1232CD90029B79
:10076300E0FEA3E0FF7C007D641203037C007D0AAE
:10077300120303ED2430FF1232CD90029BE0FEA35F
:10078300E0FF7C007D0A1203037C007D0A12030351
:10079300ED2430FF1232CD90029BE0FEA3E0FF2256
:1007A30090029BE0FEA3E0FF7C007D0A1203037C22
:1007B300007D0A120303ED2430FF1232CD90029B19
:1007C300E0FEA3E0FF7C007D0A120303ED2430FF6B
:1007D3001232CD221203037C007D0A120303ED249F
:1007E30030FF1232CD227C007D0A120303ED243048
:1007F300FF1232CD22E0FF1232CD7F2C1232CD9088
:10080300029BE4F0A3227BFF7A16797E122E5D7B96
:10081300FF221232CD90029CE004F022120303ED7A
:100823002430FF1232CD227BFF122E5D7BFF22127A
:1008330032CD90029CE004F022FF1232CD7F2C12C5
:0308430032CD2291
:1031260090029EEFF07F007E0212319990029EE09F
:08313600FD7F007E020230EF74
:102AB500E4FFFE123199E490029DF0A3F090029B91
:102AC500F0A3F090029BE0FCA3E0FDC3EC94015061
:102AD5002FA3E0FEA3E0FF74002D12279FE0FD1257
:102AE50030EF90029EE004F0700690029DE004F045
:102AF50090029CE004F070CB90029BE004F080C350
:012B050022AD
:10313E007F1F7E00123156EF64997F0160091214D1
:08314E00F775C7207F00222263
:0E324200E4F5C7F5C5F5C675C3FF75C4FF22D8
:04315600AD07AC060F
:10315A0075C78275C5011227D51227C700AFC212DB
:02316A003242EF
:01316C002240
:10319900AD07AC061227D575C78275C5031227C7B7
:0331A900023242AD
:102E3000AD07AC0675C78275C5021227D51202AB65
:102E4000F5C21227C7000DBD00010C740129F9E479
:0D2E50003AFA9002A3E014F070E002324262
:1030EF00AB07AA0675C78275C502EAF5C3AF038F92
:0C30FF00C4AF058FC21227C70002324286
:0514F70090029BEFF0E4
:1014FC00E4FFFE1231997BFF7A1679DA9002A3741D
:10150C0007F07F08122E307D097F0F1230EF7D011E
:10151C007F041230EF7F051230EF1D7F061230EF83
:10152C000D7F071230EF0DE4FF1230EF7D587F0175
:10153C001230EF7D017F101230EF7D217F111230C0
:10154C00EF7D2F7F121230EF7D3E7F131230EF12A2
:10155C0027CE7420F0E4FCEC9016E193FD600E12A3
:10156C0027B712279170031227B00C80EA12278735
:10157C0070031227B01227CE7430F0E4FCEC9016F6
:10158C00EB93FD600E1227B712279170031227B050
:10159C000C80EA12278770031227B01227CE7440F2
:1015AC00F0E4FCEC9016F593FD600E1227B71227B1
:1015BC009170031227B00C80EA1227877003122750
:1015CC00B090029BE07028A3F0A37480F0E4FCECD4
:1015DC0090171393FD600E1227B712279170031208
:1015EC0027B00C80EA12278770031227B0802612CE
:1015FC0027CE7480F0E4FCEC90173193FD600E1252
:10160C0027B712279170031227B00C80EA12278794
:10161C0070031227B07D997F1F7E001230EFE4FF1C
:03162C0002312662
:101F25000D0A2020B2BBC8CFCAB6C4E3CAE4C8EBC9
:101F3500B5C4D6B8C1EEA3ACBFC9C4DCC3BBBCD362
:101F4500BBBBD0D0C5B6A3A120A3BAA3A920200DA1
:101F55000A0D0A0041542B48454C503D310041546F
:101F65002B44454D4F3D310041542B54494D453D82
:101F75000041542B43414C4C3D0041542B53534994
:101F8500443D0041542B424541434F4E3D000D0A0F
:101F9500202D3E20C9E8D6C3B3C9B9A620202120EB
:101FA500200D0A000D0A202D3E20D6B8C1EEB4ED55
:101FB500CEF3A3A1BFC9C4DCC8B1C9D9BBD8B3B5D9
:071FC500A3A120200D0A007A
:101D0700900294E02400F582E43400F583E4F09037
:101D17000293E004F0E02407F582E43402F583E05F
:101D270022900210E024D0FFE434FFFE7C00120270
:101D3700F1AA06AB0790020FE024D0FFE434FFFEC0
:101D470022900294E02400F582E43400F5832274A3
:101D570008900293F0E4900297F0A3F022EFF0903E
:101D67000293E004F0227D0A1202F1EF2BFFEE3A14
:101D7700FE22900287E0FF2406F582E43402F58311
:101D8700E022900298E004F022900297E004F0220B
:101D97001202F1EF2BFBEE3AFA22900294F0900236
:101DA70093227B017A017902900183E0FD22900260
:0F1DB70097E0FEA3E0FFEE2290020FE024D0227F
:0300230002272091
:0D272000C0E0C083C082C0D075D000C007EB
:10272D00309906C299D2078046309843300604C2CC
:10273D0098803C7F80900207E4F0A3DFFC7F00755A
:10274D00D80075F94C75E900D2DE20980C30DFFA0F
:10275D00900287EFF0D2068016C29874072FF5828B
:0F276D00E43402F583E599F00FEFD3947F40D069
:0B277C00D007D0D0D082D083D0E03254
:102111002006030221AD900207E064C0704EA3E0E7
:10212100704A121D7964C07043EFD39411403DE4AD
:10213100900183F07F02900287E014FEEFC39E506E
:102141001C74072F121D1FFE74002FF582E4340149
:10215100F583EEF0900183E004F00F80D9121DA900
:102161001226B4121DA9121B79C20622121D79B4BE
:102171000A047E0180027E0074052FF582E4340298
:10218100F583E0B40D047F0180027F00EF5E6008FB
:10219100E4F5AF120846800FE4F5AF1204F07BFFBF
:0C21A1007A1F7925122E5DC206123286CC
:0121AD00220F
:10084600E4900299F0A3F0121D5D900299E0FEA3D8
:10085600E0FF123156900297A3121D4BEFF0900263
:100866009AE004F07006900299E004F0121D897077
:1008760003121D90C3900297E0940140CD7BFF7A4E
:100886001F795912305ABF01030204F07BFF7A1F09
:10089600796312305ABF010BE4FF1214F712329F2C
:1008A60075C7207A1F796D120B55600302098E12E7
:1008B6001D56900293121D1C640D600D121D6612CA
:1008C6001D8970EE121D9080E9121DB560030209A4
:1008D60071EF24FE602114602A14603714604E24E0
:1008E600046003020971121DBFFEE434FF900295F5
:1008F600F0A3CEF0020978121D3C7C007D0A12029C
:10090600F180277D0A121D287D64121D6F90021149
:1009160002095C7D64121D287C037DE8121D9790F8
:100926000211121D3F7C00121D6DA380299002103A
:10093600121D3F7C037DE8121D357C277D10121D9C
:1009460097900211121D3F7C007D64121D97A31221
:100956001D3F121D6DA3E024D0FDEC34FFCD2FFF0B
:10096600ED3E900295F0A3EFF08007E4900295F03B
:10097600A3F0900295E0FCA3E0FDEC900000F0A34C
:10098600EDF0122AB512329F7A1F7976120B557046
:1009960074121D56900293121D1C640D600D121DDB
:1009A60066121D8970EE121D9080E9D3900298E0C0
:1009B6009406900297E0940040031232AB9002979F
:1009C600E07002A3E070031232AB7408121DA1F0AE
:1009D600900298E02408FF900297E03400FE90020F
:1009E60093E0FDC39FE49E501674072D121D1FFF52
:1009F600121D48EFF0900294E004121D6580D1129A
:100A06001D48120B5E7BFF7A1F797F12305AEF6406
:100A160001704B121D56900293121D1C640D600D41
:100A2600121D66121D8970EE121D9080E9121DB509
:100A36007020EF24FE6008047018121DBF800D128E
:100A46001DBF75F00AA4FFA3E024D02F90000FF07D
:100A5600800690000F740AF0122AB512329F7BFFAF
:100A66007A1F798812305AEF64016003020B5474BE
:100A76000A121D58900293121D1CFF640D6011EF9F
:100A8600B42C08121D897003121D90121D6680E495
:100A9600900297E07004A3E0640660030232AB9014
:100AA6000293740A121D1B24D0900010121D1564A7
:100AB6002C60031232AB121D16900011121D156424
:100AC6002C60031232AB7420121DA1801290029387
:100AD600121D1CFF642C600C121D48121D64A3E03D
:100AE60004F080E9121D07900012121D15642C6097
:100AF600031232AB9002947430F0900293801290FD
:100B06000293121D1CFF642C600C121D48121D64FA
:100B1600A3E004F080E9121D07900013121D15646E
:100B26002C60031232AB9002947440F090029380D2
:100B360012900293121D1CFF640D600C121D4812C8
:0E0B46001D64A3E004F080E9121D48120B5E4E
:100B5400227BFF12305AEF640122E4F0122AB5120C
:030B6400329F229B
:0C329F001204F07BFF7A1F7993022E5D71
:0C32AB001204F07BFF7A1F79A9022E5D4F
:10305A00E4FF1202ABFE601674072F121D1F6E608A
:10306A00037F00220F740129F9E43AFA80E47F0110
:01307A002233
:0F31CE00759850759CFD758E11758911023183AE
:10318300C2ACC206E4900287F07F80900207E4F0AD
:05319300A3DFFCD2AC3B
:013198002214
:102E5D0090029FEBF0A3EAF0A3E9F090029FE0FB54
:102E6D00A3E0FAA3E0F91202ABFF600F1232CD908E
:0C2E7D0002A0E475F00112035880E0226E
:0A32CD00C2078F993007FDC20722E7
:10186E000F90028BE0FBA3E0FAA3E0F98F82758361
:10187E00000202C4FD74182EF582E43403F583EDE4
:10188E00F00E0F2290028BE0FBA3E0FAA3E0F92208
:10189E0090028CE0900304F090028DE0900305F02E
:1018AE0090028EE0900306F090028FE0900307F016
:1018BE009002902290028DE0900304F090028EE050
:1018CE00900305F090028FE0900306F0900290E0F6
:1018DE00900307F090029122FD740E2EF582E434EF
:1018EE00032290028CE0900305F090028DE09003AD
:1018FE0006F090028EE0900307F090028F22900285
:10190E008BE0248CF582E43402F583EEF090028BAA
:10191E00E004F00F22EBF0A3EAF0A3E9F0E422904A
:10192E00028CE0900306F090028DE0900307F09099
:10193E00028E22F09002FFE0FFA3E0900322CFF090
:10194E00A3EFF07F012290028EE024D022748E2D20
:10195E00F582E43402F583EFF00C0D22C294C2003E
:10196E00D28022FFE434FFFE7C007D0A0202F19059
:0B197E00028CE0900307F090028D2225
:102DCD0020932E7F017E0012307B209324900325CB
:102DDD00E004F0E0D394044002E4F0900325E0FF1A
:102DED001231263093FD7F017E0012307B3093F33C
:022DFD00222290
:10295D00122DCD900325E024FE6015146033146014
:10296D0033240370339003247401F0D294022E8922
:10297D00900324E064026003122DFF90032474027F
:10298D00F0D294300222C20230001D122BDEC200A2
:10299D00220229B612196A22E4900324F02094052C
:0929AD00123286D294122EE022AF
:102DFF00E4FFFE123156EF7F00FEC006C0070F7EC4
:102E0F0000123156EFFDD0E02DFFD0E03400FE90E0
:102E1F000326F0A3EFF0900301EEF0A3EFF0C20250
:012E2F002280
:1029B600900324E0640360097403F012196A122D6F
:1029C600FF300242C202123286D294E4900293F0A1
:1029D600A3F02000287F147E0012307B900294E042
:1029E60004F07006900293E004F0D3900294E09411
:1029F6002C900293E0940140D912196A22122BDE20
:062A060012196A122DFFF7
:012A0C0022A7
:1023F700900325E024FE601214601714602524035F
:102407007029D281D282B2838027B281D282D283CD
:10241700801FD283308206C282C2818014D282D2C8
:1024270081800ED281B282D2838006D282D283D2B9
:1024370081900326E0FEA3E0FF4E601F900302E0B9
:1024470024FFF0900301E034FFF0E07002A3E07096
:102457000A900301EEF0A3EFF0D20290030CE00420
:10246700F0700690030BE004F0D390030CE09404A3
:0F24770090030BE094004006E4F0A3F0D20122A2
:102EE0003091037F00227F017E0012307B309103FE
:102EF0007F00223091FD7F017E0012307B3091F304
:0B2F0000300005122BDEC2007F012212
:102E890030000D122486BF0107122BDEC20080120A
:102E990030011830000C122B53BF0106122BDEC271
:0C2EA9000022E490030BF0A3F0C2012211
:102F8900E4900322F0A3F090030DF0C20090032413
:102F9900F0122DFFE490030BF0A3F0FF7E02123133
:072FA90056900325EFF02212
:031A8F009002883A
:101A9200121923FFFE900288121872FD6009B42CFD
:101AA200010E0FEEB409EE900288121872642D70C6
:101AB200600F90028BF0900288121872FE642E6002
:101AC2000512190C80F07F069003037430F0A3DF37
:101AD200FC900303742DF090028BE024FE6013143B
:101AE20060151460171460192404701A90028C0295
:101AF2001B0B12197D801212192D800D1218F08005
:101B02000812189E80031218C2E0900308F0021B0C
:101B120073E490028BF0900288121872FE642E60B9
:101B22000512190C80F07F069003037430F0A3DFD6
:101B3200FC90028BE024FE601314601614601814EB
:101B4200601A2404701B90028C021B6E12197D0213
:101B52001B6E12192D80151218F0801012189E801B
:101B62000B90028CE0900303F01218C2E09003087D
:061B7200F0E4900309F00D
:011B7800224A
:032C660090028851
:102C6900121923FFFE900288121872FD6009B42C14
:102C7900010E0FEEB402EE900288121872B44119D7
:102C89007B017A017985121DC67B017A017985124A
:0F2C99001989C280D2007F0122B280C2007F0061
:012CA8002209
:031DC60090028BFD
:101DC900121923FFFE12186F6009B42C010E0FEED1
:101DD900B403F2E4FE12186FFD642E600512188335
:101DE90080F390028B12189512188312187A121820
:101DF9008212187A12188212186F642C60030F80ED
:101E0900F612186E12188274182EF582E43403F54E
:101E190083E4F012186F642C60030F80F60FE4FE60
:101E290012186FFD642E60081218E712188B80F0E3
:101E390090028B1218951218E712188B12187A1241
:101E490018E612188B12187A1218E612188B121843
:101E59006F642C60030F80F612186E1218E6F58372
:0C1E6900EDF00E1218E7F583E4F07F01A5
:011E7500224A
:1024860090030AE07002FF22900322E0FEA3E0FF21
:102496009002FFE0FAA3E0FBD39FEA9E4008EB9F81
:1024A600FDEA9EFC80159002FFE0FEA3E0FFC390CC
:1024B6000323E09FFD900322E09EFCD3ED94B4EC51
:1024C6009400401074689D900294F074019C9002F0
:1024D60093F08008900293ECF0A3EDF0D390029471
:1024E600E09419900293E094004008E490030D12E2
:0524F6001941227F00E6
:0124FB0022BE
:102B530090030AE0FE7002FF2290030DE004F0EE02
:102B6300C3940A500AE0940B400280227F00229013
:102B7300030AE0C39432500D90030DE09407400222
:102B8300800C7F002290030DE0D394054005E412EE
:062B93001941227F00221F
:0319890090028B3E
:10198C00121923FCFD1218928C8212187C6009B477
:10199C002C010D0CEDB407ED1218928C8212187CF0
:1019AC00B42C03E4804BE4FD1218928C8212187C48
:1019BC00FF642E600512195B80EEED24FD601204AD
:1019CC00702C12195475F00AA4FFA3E024D02F80B8
:1019DC002090028FE024D075F00AA4FF12195475E0
:1019EC00F064A42FFF900290E024D02F80031219F2
:1019FC005490030AF01218928C8212187C642C609A
:101A0C00030C80F10C1218928C8212187CB42C08E6
:101A1C00E49002FFF0A3F022E4FD1218928C8212E3
:101A2C00187CFF642E600512195B80EEED24FD60BE
:101A3C000C047040121954121971A3802390028F58
:101A4C00E024D0121971AA06AB07121954FFE43422
:101A5C00FFFE7D641202F1EF2BFFEE3AFE90029036
:101A6C00E024D0FDEC34FFCD2FFFED3E9002FFF0D3
:101A7C00A3EFF022121954FEE434FF9002FFF0A3FE
:021A8C00CEF09A
:011A8E002235
:0E325000244750524D43002447504747410049
:102FF600A3F07B017A01798522900206E02485F50B
:1030060082E43401F58322E0FBA3E0FAA3E0F902AF
:0230160002AB0B
:03004300021C4656
:101C4600C0E0C0F0C083C082C0D075D000C000C064
:101C560001C002C003C004C005C006C007E59A3033
:101C6600E106539AFD021CECE59A30E079539AFEA0
:101C7600122FFFE59BF0900206E004F0900184E04D
:101C860004F0E59B640A7053122FFFE4F0900206FD
:101C9600E004F0200A2190028B74FFF0A37432F066
:101CA6007450122FF6122D25EF64017027122FF8AB
:101CB600122C66D20A801D90028B74FFF0A3743238
:101CC600F07457122FF6122D25BF0108122FF812A5
:101CD6001A8FC20A900206E4F0800B900206E0D347
:101CE600947E4002E4F0D007D006D005D004D0039D
:101CF600D002D001D000D0D0D082D083D0F0D0E0B6
:011D060032AA
:102D2500900288EBF0A3EAF0A3E9F090028B123051
:102D35000DFF602290028812300D6F60037F002224
:102D4500900289E475F00112035890028CE475F045
:092D55000112035880D57F012210
:0632E500759A50023286CA
:0D328600E4F5AFC200900206F075AF012222
:102F0B00E4F5D875F9FDF5E9D2DE22C313F0448060
:102F1B00F0900182E004F022C2ACE4F5AFD2C2D251
:0B2F2B0080D29022900100E06403229D
:1028A60020B559122F23121FCC900293EFF012314C
:1028B60083123286900293E064017040122F28C280
:1028C600C27FC01232CDE4FF1232CDE4900294F002
:1028D600900183E0FF900294E0FEC39F50177402BC
:1028E6002EF582E43401F583E0FF1232CD90029496
:0C28F600E004F080DB7FC01232CDD2C2C3
:0129020022B2
:0E1B7900900296EBF0A3EAF0A3E9F0A3EDF0E2
:101B8700122F23C290C2B6D2B7D295D2B390018298
:101B9700F0900325E0700D90029AF0121C2C944CE3
:101BA70040F9800CE490029AF0121C2C947240F9D0
:101BB700E490029AF0900299E0FFA3E0C39F5024BB
:101BC700900296E0FBA3E0FAA3E0F91202ABFF1242
:101BD7002848900297E475F00112035890029AE0A2
:101BE70004F080D1900348E0FF122848900347E0B3
:101BF700FF122848900325E0700F90029AF0121CFC
:101C07003AE0C3940540F7800EE490029AF0121C64
:101C17003AE0C3940A40F7D2B6C2B7C295D290123F
:051C270031830232864A
:101C2C007F7E12284890029AE004F0E0C3227F7E67
:0A1C3C0012284890029AE004F022FA
:101FCC00122072122F2F60037F0022900101E0B4C7
:101FDC007E0B12256B122F2F60F17F0022E49002F2
:101FEC0095F0900101E0FF647E602C900295E02456
:101FFC0002F582E43401F583EFF0900295E004F0F1
:10200C0012256B900295E0D3947840037F00221246
:10201C002F2F60CE7F00227B017A017902900295EE
:10202C00E024FEFD1226B4900295E0FE2400F58219
:10203C00E43401F583E0FF900348E06F60037F0018
:10204C002274012EF582E43401F583E0FF900347FE
:10205C00E06F60037F0022900295E024FEF0E09098
:05206C000183F07F017B
:01207100224C
:10207200E4900100F01232D71232D7E4900101F05D
:1020820030B40A30B5FA9001007401F02220B40A8B
:1020920030B5FA9001007402F022A2B49204E490E6
:1020A2000182F0900296F01231EC900101E0C3132C
:1020B200F0900182E0B40616900296E004F0E0B4DB
:1020C200030C9001007403F0E4900182F022E4908A
:1020D2000182F0C2052005CF122F0B20DF1C30B584
:1020E200079001007404F022A2B4300401B350EB53
:1020F200A2B49204D205D2DF80E12005D89001017A
:0E210200E0122F16E0B407CD9001007405F036
:0121100022AC
:10256B00E4900296F0900296E0C394085060122F0C
:10257B000B20DF2030B5079001007404F022A2B4C9
:10258B00300401B3500AA2B49204D205D2DF80E129
:10259B00C20580DD200515900101E0FF122F16E02A
:1025AB00B407079001007405F022801A1231EC90E9
:1025BB000182E0B40504E4F080AB900101E0C313A9
:0E25CB00F0E4900182F0900296E004F0809718
:0125D90022DF
:0528480090029BEFF07F
:10284D00BF7E04D2038002C203E490029CF090028A
:10285D009BE054017004B2B38023122F1C2003049B
:10286D007F0180027F00900182E0B405047E01802B
:10287D00027E00EE5F600A1231DDB2B3E490018298
:10288D00F090029BE0FFC313F01231DD90029CE04B
:08289D0004F0E0C3940840B60A
:0128A5002210
:0F31DD00E4F5D875F9FD75E908D2DE30DFFD2283
:0732D700122F0B30DFFD2276
:0F31EC00E4F5D875F9FE75E980D2DE30DFFD22FB
:0732DE00C295D2B6C2B7226F
:10119300000011892312329B462457AD653674BF74
:1011A3008C489DC1AF5ABED3CA6CDBE5E97EF8F724
:1011B300108101083393221A56A5472C75B7643E54
:1011C3009CC98D40BFDBAE52DAEDCB64F9FFE87604
:1011D3002102308B02101399672676AF443455BD34
:1011E300AD4ABCC38E589FD1EB6EFAE7C87CD9F5E4
:1011F3003183200A1291031877A7662E54B5453C14
:10120300BDCBAC429ED98F50FBEFEA66D8FDC974C3
:101213004204538D6116709F042015A9273236BBF3
:10122300CE4CDFC5ED5EFCD7886899E1AB7ABAF3A3
:101233005285430C7197601E14A1052837B3263AD3
:10124300DECDCF44FDDFEC5698E98960BBFBAA7283
:101253006306728F4014519D252234AB063017B9B3
:10126300EF4EFEC7CC5CDDD5A96AB8E38A789BF163
:101273007387620E5095411C35A3242A16B1073893
:10128300FFCFEE46DCDDCD54B9EBA8629AF98B7043
:1012930084089581A71AB693C22CD3A5E13EF0B773
:1012A300084019C92B523ADB4E645FED6D767CFF23
:1012B30094898500B79BA612D2ADC324F1BFE03653
:1012C30018C109483BD32A5A5EE54F6C7DF76C7E03
:1012D300A50AB48386189791E32EF2A7C03CD1B533
:1012E300294238CB0A501BD96F667EEF4C745DFDE3
:1012F300B58BA40296998710F3AFE226D0BDC13413
:1013030039C3284A1AD10B587FE76E6E5CF54D7CC2
:10131300C60CD785E51EF497802891A1A33AB2B3F2
:101323004A445BCD695678DF0C601DE92F723EFBA2
:10133300D68DC704F59FE41690A98120B3BBA232D2
:101343005AC54B4C79D7685E1CE10D683FF32E7A82
:10135300E70EF687C41CD595A12AB0A3823893B1B2
:101363006B467ACF485459DD2D623CEB0E701FF962
:10137300F78FE606D49DC514B1ABA02292B9833092
:101383007BC76A4E58D5495C3DE32C6A1EF10F7842
:0526B400900296EDF01C
:1026B90074FFA3F0A3F0900296E0D39400403F1278
:1026C90002ABFF900297A3E06F25E0FFE433FE74AD
:1026D900932FF58274113EF583E493FC740193FD05
:1026E900900297E0FFECFEED6FFFEEF0A3EFF090A4
:1026F9000296E014F0740129F9E43AFA80B89002DC
:1027090097E0FEA3E0F4FFEEF4FCEF900348F0AE8F
:0627190004EE900347F0FE
:01271F002297
:0E325E0057494445312000574944453220006D
:102A62001FEF25E0FF74022EF582E43401F583EDB9
:102A720054E1F074022EF582E43401F58322742EBF
:102A82002FF582E43403F58322F0900329E004F069
:102A920022EE75F007A414F0AF067BFF227B017AC9
:102AA200017902900183E0FD2290032CE4F0A374EB
:032AB20008F02207
:1031AC0090010FE020E00B1222D7EF6401600312B4
:0331BC0023672264
:1022D7009003497403F07F057E00123156EF6401C5
:1022E700707B900349E0FED3940840037F0022905F
:1022F700034A122A937A32795E122CEBEF6401704B
:102307004390034AE0FE2402122A78E0FD541EC3DC
:1023170013FF7002FF22122A62E04FF0EF700D9058
:10232700034AE02402122A78E04480F07F077E0007
:10233700123156BF0108900349E0FF12174F1231BF
:10234700FB7F012290034AE02402122A78E030E062
:0F235700037F0022900349E004F00222E97F0097
:012366002254
:1023670090034B7403F07F067E00123156EF640131
:10237700707B90034BE0FED3940840037F002290CC
:10238700034C122A937A327965122CEBEF640170B1
:102397004390034CE0FE2402122A78E0FD541EC34A
:1023A70013FF7002FF22122A62E04FF0EF700D90C8
:1023B700034CE02402122A78E04480F07F077E0075
:1023C700123156BF010890034BE0FF12174F12312D
:1023D700FB7F012290034CE02402122A78E030E0D0
:0F23E700037F002290034BE004F00223797F0074
:0123F60022C4
:102CEB00EF1475F007A490034EF01202AB60282589
:102CFB00E0FFE433FE90034EE02402122A78E06FEB
:102D0B007001EE60037F0022740129F9E43AFA9016
:092D1B00034EE004F080D37F01B7
:012D2400228C
:05174F00900328EFF0FB
:10175400900183E0D39478400302186D122AABFF02
:101764007E00123156EF700302186D122AABE4901A
:101774000329F0900329E0FFC39406500A122A803B
:101784007440122A8B80ECE4900329F090032CE03F
:10179400FEA3E0FF12315690032BEFF06029900373
:1017A4002BE025E0FF900329E0242E122A83EFF09A
:1017B40090032DE004F0700690032CE004F0122A4C
:1017C4008CE0C3940640C57F0F7E00123156EF258E
:1017D400E044E0900334F090032AE004F0900183A5
:1017E400E0FF90032BF0900328E075F007A424F8A1
:1017F400FEC3EF9E90032AF0E4900329F090032A9D
:10180400E0FF900329E0C39F502290032BE0FF24C4
:1018140002122A78E0FE74092FF582E43401F5837C
:10182400EEF090032BE014122A8B80D1900328E071
:101834001475F007A490032BF0E4900329F09003AF
:1018440029E0FFC39407501A122A80E0FF90032B6B
:10185400E02402122A78EFF090032BE004122A8B82
:0918640080DC900183E02407F010
:01186D002258
:0F31FB0030B5FD122A9F1226B4122A9F021B79AB
:10004600EC4D6011E8497017ED33EC3304600DE4B4
:10005600FCFFFEFD22E933E8330470F80202961233
:10006600026158046009E4CC248150062850090234
:1000760002A028400302029DC0E0EB4A7044B9800A
:1000860006D0E0FB02028CEF4E701CBD8008EBFF31
:10009600EAFEE9FD80EBE98DF0A4FEE5F002012F12
:1000A600E9CDF9EAFEEBFFEF89F0A4FCE5F0CE8995
:1000B600F0A42EFFE435F0CD89F0A42DFEE435F052
:1000C6008067EF4E7005BD80D780C3EF8BF0A4AC80
:1000D600F0EE8BF0A42CFCE435F0F8EF8AF0A42CBB
:1000E600E5F038FCE433CB8DF0A42CFCE5F03BF8CE
:1000F600EE8AF0A42CFCE5F038F8E433CF89F0A4BE
:100106002CFCE5F038CF3400CE89F0A42FFFE5F0C3
:100116003EFEE433C98DF0A42EFEE5F039CD8AF01B
:10012600A42FFFE5F03EFEE43DFD33D0E0FB500793
:100136000BBB000F0202A0EC2CFCEF33FFEE33FEEC
:06014600ED33FD0202781A
:10014C000202A0EC5D046005E859047003020296FB
:10015C00120261580460F6EC4860F2EC7004FDFE8B
:10016C00FF22C860DB2481C85009C3986002500686
:10017C0002029D9850CAF582E9294B4A7005AB8260
:10018C0002028C75F0007C1A7880C3EF9BEE9AED1E
:10019C0099400DC3EF9BFFEE9AFEED99FDE842F0FE
:1001AC00DC23ACF0D0E0FFD0E0FED0E0FDAB822051
:1001BC00E7101BEB60BAEC2CFCEF33FFEE33FEEDDB
:1001CC0033FD020278E803F830E705C0F075F00063
:1001DC00EF2FFFEE33FEED33FD40B830E7C280AABF
:1001EC0075F020800E75F010800575F0087D007E8E
:1001FC00007F003392D530D50312048BEC334010C2
:10020C00EF33FFEE33FEED33FDEC33FCD5F0ED2296
:0E021C00E5F0247EA2D513CC92E7CDCEFF22D2
:10022A00EDD2E7CD33EC3392D524814006E4FFFECC
:10023A00FDFC22FCE4CFCECDCC24E0501174FF802B
:10024A00EDC3CC13CCCD13CDCE13CECF13CF0470C8
:07025A00F030D5DE02048B39
:10026100E9D2E7C933E833F892D5EDD2E7CD33ECE3
:0702710033FC5002B2D5225C
:10027800EC30E7100FBF000C0EBE00080DBD0004E7
:100288000BEB6014A2D5EB13FCED92E7FD2274FF93
:10029800FCFDFEFF22E480F8A2D574FF13FC7D80EC
:0302A800E480EF00
:030000000232B712
:0C32B700787FE4F6D8FD7581210230D349
:1002AB00BB010689828A83E0225002E722BBFE0251
:0902BB00E32289828A83E4932284
:1002C400BB010CE58229F582E5833AF583E02250EF
:1002D40006E92582F8E622BBFE06E92582F8E22239
:0D02E400E58229F582E5833AF583E4932253
:1002F100EF8DF0A4A8F0CF8CF0A428CE8DF0A42E21
:02030100FE22DA
:10030300BC000BBE0029EF8DF084FFADF022E4CCDE
:10031300F875F008EF2FFFEE33FEEC33FCEE9DECA7
:10032300984005FCEE9DFE0FD5F0E9E4CEFD22EDED
:10033300F8F5F0EE8420D21CFEADF075F008EF2F37
:10034300FFED33FD4007985006D5F0F222C398FD28
:050353000FD5F0EA22C5
:10035800C5F0F8A3E028F0C5F0F8E5821582700230
:060368001583E038F022CD
:10036E00E88FF0A4CC8BF0A42CFCE98EF0A42CFC2E
:10037E008AF0EDA42CFCEA8EF0A4CDA8F08BF0A4AC
:10038E002DCC3825F0FDE98FF0A42CCD35F0FCEB0B
:10039E008EF0A4FEA9F0EB8FF0A4CFC5F02ECD39D0
:0F03AE00FEE43CFCEAA42DCE35F0FDE43CFC223D
:1003BD0075F008758200EF2FFFEE33FECD33CDCCF7
:1003CD0033CCC58233C5829BED9AEC99E58298407A
:1003DD000CF582EE9BFEED9AFDEC99FC0FD5F0D657
:1003ED00E4CEFBE4CDFAE4CCF9A88222B800C1B981
:1003FD000059BA002DEC8BF084CFCECDFCE5F0CBBF
:10040D00F97818EF2FFFEE33FEED33FDEC33FCEBF7
:10041D0033FB10D703994004EB99FB0FD8E5E4F9B2
:10042D00FA227818EF2FFFEE33FEED33FDEC33FC9F
:10043D00C933C910D7059BE99A4007EC9BFCE99A93
:10044D00F90FD8E0E4C9FAE4CCFB2275F010EF2FD8
:10045D00FFEE33FEED33FDCC33CCC833C810D707D8
:10046D009BEC9AE899400AED9BFDEC9AFCE899F813
:0E047D000FD5F0DAE4CDFBE4CCFAE4C8F922A6
:102C2200C2D5E830E70FB2D5E4C39BFBE49AFAE4DD
:102C320099F9E498F8EC30E717B2D5122C58120340
:102C4200F9E4C39BFBE49AFAE499F9E498F8800367
:102C52001203F930D50DE4C39FFFE49EFEE49DFD0F
:042C6200E49CFC22D0
:0E048B00C3E49FFFE49EFEE49DFDE49CFC2282
:10049900EB9FF5F0EA9E42F0E99D42F0E89C45F0B9
:0104A9002230
:1004AA00E8600FECC313FCED13FDEE13FEEF13FF30
:0304BA00D8F12254
:1004BD00E86010ECA2E713FCED13FDEE13FEEF1355
:0404CD00FFD8F02242
:1004D100E8600FEFC333FFEE33FEED33FDEC33FC89
:0304E100D8F1222D
:0C04E400ECF0A3EDF0A3EEF0A3EFF0228B
:00000001FF
